:020000040000FA
:020000000428D2
:08000800FF30A2001121AA0142
:10001000AB01AC01AD01E630AE00AF01831601309B
:100020009F00831207309900FF301F2122111E21EB
:1000300022121D21A2121C21231118212312172183
:10004000A3121621013024210130A400A408031DAD
:100050002A284928B001A0102011D52083161E0897
:10006000A70083121E08A60001302B21B001A010AA
:100070002011D52083161E08AD0083121E08AC0087
:100080002608B0002708B1002C08B2002D08BC20BB
:1000900026280130A8002630A9000130B000D53054
:1000A000B1002C08B2002D08BC202408023C031D1E
:1000B0005D280130A800B930A9000230B0009130AD
:1000C000B1002C08B2002D08BC202408023C031DFE
:1000D0006D280230A8004C30A9000330B0004D302C
:1000E000B1002C08B2002D08BC202408023C031DDE
:1000F0007D280230A800E030A900AF01B001A010B7
:100100002011D52083161E08AA0083121E08AB00FA
:1001100085188B2888282808B0002908B1002B08EA
:10012000B2002A08BC202408023C031D9928A520FF
:10013000A328A52001302E02AE0046302E0203185F
:10014000A3284630AE007E28A42823151821A50137
:100150002E082502031CAD28B62800000000000070
:10016000A50A8518B528FA30A500A828231118215A
:10017000851CBB28B8280800B3003208B002031958
:10018000C4280318CE28D1283308B1020319CB287C
:100190000318CE28D1280030A40008000130A400A4
:1001A00008000230A40008000800B008031DDB2886
:1001B0000130B100EF283008013C031DE228023075
:1001C000B100EF283008023C031DE9280430B100DB
:1001D000EF283008033C031DEF280830B1008316D8
:1001E0003108103E9F0083123008B3000230B40083
:1001F00051213508B2003208B00030089F00A01C21
:1002000003291F1704291F13201D08299F130929DB
:100210009F171F14323044219F149F1C10290D2951
:1002200008008316FF23900083120800192919295A
:100230001929230885000800212921292129A20044
:100240002129220865000800B0003008B1006430A0
:10025000B20064303229B0003008B1006430B2001E
:100260000A303229B300FF30B4003208B60031083A
:10027000B5001730340703183A29B50B3929B60BE6
:100280003729B30B35290800B300F430B400FC3033
:10029000B50033083407031C0034350703184D2913
:1002A00008003408003C031C56295C290310B30DD8
:0E02B00001303402B40051293308B5000800B3
:02400E0084111B
:00000001FF
